:1000000050C0000068C0000066C0000064C000006E
:1000100062C0000060C000005EC000005CC0000064
:100020005AC0000058C0000056C0000054C0000074
:1000300052C0000050C000004EC000004CC0000084
:100040004AC0000048C0000046C0000044C0000094
:1000500042C0000040C000003EC000003CC00000A4
:100060003AC0000072C5000036C0000034C0000075
:1000700032C0000030C000002EC000002CC00000C4
:100080002AC0000028C0000026C0000024C00000D4
:1000900022C0000020C000001EC000001CC00000E4
:1000A000DB0511241FBECFEFCDBFDFE3DEBF2CE3A6
:1000B000A0E0BCE301C01D92A838B207E1F710E050
:1000C000C1E5D0E003C02197FE011BD7C035D107A1
:1000D000D1F78BD531C794CF90E0FC01EE52F04BB5
:1000E00020812F3F51F08755904BDC01EC91B0E21D
:1000F000EB9FF0011124FC5F218308958091433C24
:10010000811117C01092443C1092453C1092463C1D
:100110001092473C1092483C1092493C10924A3C45
:1001200010924B3C10924C3C10924D3C81E08093DD
:10013000433C8091E3058C7F9091423C892B8093D6
:10014000E305911117C084E0C7DF86E0C5DF809129
:10015000C10884608093C1088091C0088162809347
:10016000C00890917D3C80917E3C9093C008809324
:10017000C1080895913021F48EE0AEDF80E1E6CF32
:10018000923029F78EE1A8DF80E2E0CF0000809373
:10019000C4088091C30887FFFCCF8091C4080895EC
:1001A000282F30E0F901EE52F04B40814F3F09F427
:1001B00050C0893258F4F901E95AF04BE081EE233E
:1001C00029F0E13099F010F0E63020F1F901E7551F
:1001D000F04BE081A0E2EA9FF0011124FC5F8081F6
:1001E000842321F1611120C046830895F901E0586C
:1001F000F04B5081533008F05F5F7091010A81E04D
:1002000090E001C0880F5A95EAF780958723809384
:10021000010ADCCF80E1E89FF0011124E05AF54F9C
:1002200081818F7E8183D2CF458308952058304BC2
:10023000D9018C91309771F08F3F61F07096E80F83
:10024000F11D9FB7F8948081611107C0877F80837B
:100250009FBF0895F0E0E0E0F4CF8860F8CF8FB75B
:10026000F8942091103C3091113C4091123C5091F7
:10027000133CE091AA0AF091AB0A9091A60A90FF74
:1002800008C02F5F3F4F4F4F5F4FE091AA0AF09198
:10029000AB0A8FBFA8EEB3E001D623E0F695E79551
:1002A0002A95E1F76E0F7F1F811D911D08958F9292
:1002B0009F92AF92BF92CF92DF92EF92FF924B014B
:1002C0005C01CDDF6B017C01A8EEB3E0A5019401D8
:1002D000E5D5C60ED71EE81EF91EC616D706E806D7
:1002E000F90610F4BCDFF9CFBADF6C157D058E0579
:1002F0009F05D0F3FF90EF90DF90CF90BF90AF902D
:100300009F908F9008958F929F92AF92BF92CF92BD
:10031000DF92EF92FF920F93CF93DF93FC018081E6
:10032000893210F461E03CDF8091443C882319F06D
:1003300081FF0DC07894DF91CF910F91FF90EF90E6
:10034000DF90CF90BF90AF909F908F90089580FFE7
:10035000F2CF8090463C9090473CA090483CB090B3
:10036000493CC12CD12C7601E0E09401A501B601F5
:10037000C701A0E0BAD581F1217030E040E050E043
:1003800060E070E080E090E0B0D5D1F0B0E0A0E0B7
:10039000E03370F4AE2FA695A695A695F0E2AF9F38
:1003A000D0011124A05FBB4F8E2F8770A80FB11D05
:1003B000CE2FD0E0C25CD34C88899C91892B8C9342
:1003C0009401A501B601C70101E074D549015A01A4
:1003D0006B017C01EF5FC9CF80904A3C90904B3C11
:1003E000A0904C3CB0904D3CC12CD12C7601E0E269
:1003F0009401A501B601C701A0E077D509F49BCF10
:10040000217030E040E050E060E070E080E090E09B
:100410006CD5D1F0B0E0A0E0E03370F4AE2FA6953B
:10042000A695A69580E2A89FD0011124A05FBB4F9E
:100430008E2F8770A80FB11DCE2FD0E0C25CD34C99
:1004400088899C91892B8C939401A501B601C701E1
:1004500001E030D549015A016B017C01EF5FC8CF43
:100460006F927F928F929F92AF92BF92CF92DF92C4
:10047000EF92FF920F93CF93DF933C018091443C26
:10048000882319F081FF1BC0F89481E38093C00892
:1004900084E08093C108F3018081893208F09CC018
:1004A00060E0DF91CF910F91FF90EF90DF90CF90C0
:1004B000BF90AF909F908F907F906F9071CE80FF94
:1004C000E4CF8090463C9090473CA090483CB09050
:1004D000493CC12CD12C7601B0E09401A501B601B4
:1004E000C701A0E002D591F1217030E040E050E07A
:1004F00060E070E080E090E0F8D4E1F0D0E0C0E0AF
:10050000B03370F4CB2FC695C695C69580E2C89FD0
:10051000E0011124C05FDB4F8B2F8770C80FD11D06
:100520008B2F90E02881825C934CFC01208B88818A
:10053000887F88839401A501B601C70101E0BAD480
:1005400049015A016B017C01BF5FC7CF80904A3CD3
:1005500090904B3CA0904C3CB0904D3CC12CD12C89
:100560007601B0E29401A501B601C701A0E0BDD4B7
:1005700009F48BCF217030E040E050E060E070E0A3
:1005800080E090E0B2D4E1F0D0E0C0E0B03370F4AD
:10059000CB2FC695C695C695F0E2CF9FE0011124FA
:1005A000C05FDB4F8B2F8770C80FD11D8B2F90E062
:1005B0002881825C934CFC01208B8881887F888312
:1005C0009401A501B601C70101E074D449015A01A3
:1005D0006B017C01BF5FC6CFDF91CF910F91FF9080
:1005E000EF90DF90CF90BF90AF909F908F907F90D3
:1005F0006F900895FF920F931F93CF93DF93EC01B9
:10060000F62E042F122F2CDF85E0C0DD8F2DBEDDEE
:10061000802FBCDD812FBADDCE01DF91CF911F91FC
:100620000F91FF9070CEDF92EF92FF920F931F9386
:10063000CF93DF937C01C62FD42E152F022F10DF0E
:1006400082E0A4DD8C2FA2DDCD2DD12F0C0F1D2F2C
:10065000111DC017D10719F0899198DDFACFC70194
:10066000DF91CF911F910F91FF90EF90DF904BCED4
:100670000F931F93CF93DF93EC01062F142FF0DE1F
:1006800082E084DD802F82DD812F80DDCE01DF914D
:10069000CF911F910F9137CE1F93CF93DF93EC0132
:1006A000162FDEDE83E072DD812F70DD80E06EDDEF
:1006B000182FCE0128DE812FDF91CF911F91089551
:1006C000CF92DF92EF92FF921F93CF93DF93EC01D3
:1006D000162F262F40EE6FE08DDF8FB7F894C09075
:1006E000103CD090113CE090123CF090133C8FBF36
:1006F0008AE0C80ED11CE11CF11C2FB7F894809140
:10070000103C9091113CA091123CB091133C2FBF32
:100710008C159D05AE05BF0590F46EE0CE01BCDFE3
:10072000807E1813EACF81E091E0892790E0DF9185
:10073000CF911F91FF90EF90DF90CF90089580E0D0
:10074000F3CF0F931F93CF93DF93EC0160E8B8DFF3
:100750008C01892B61F440E06AE2CE0189DF40E937
:1007600069E2CE0185DF42E868E2CE0181DFC8019F
:10077000DF91CF911F910F91089560E0A1CF7F92FB
:100780008F929F92AF92BF92CF92DF92EF92FF92A1
:100790000F931F93CF93DF93CDB7DEB7A297CDBF53
:1007A000DEBF8C015DDE80ECF1DCC801ACDD6AE00F
:1007B00070E080E090E07BDDCE0101967C018EE070
:1007C000F70111928A95E9F72EE0A70160E3C801CD
:1007D0002ADF2EE0A70160E4C80125DF2EE0A70193
:1007E00060E5C80120DF40E060E6C80141DF40E08D
:1007F00060E7C8013DDF43EA6BE2C80139DF24E06E
:1008000047E660E6C801F6DE21E047E660E7C8019A
:10081000F1DE8CE0ECE3FFE4DE011F9601900D9227
:100820008A95E1F74E01FFE08F0E911CB12CA12CAF
:1008300028E0722EF401E190F1904F0160E8C801C8
:100840003FDF6C01892B09F065C0F2E0EF16F1047F
:1008500009F472C058F4E114F10409F473C0EA9485
:10086000EF2889F0CC24C394D12C54C0E4E0EE16D8
:10087000F10409F465C008F461C085E0E816F104EC
:1008800089F768E101C064E091E0A916B10409F0BC
:100890005BC01E8E1D8E7C8E1B8E24E0AE01455EDD
:1008A0005F4FC801C0DEEFEFAE1ABE0AF6E0AF162A
:1008B000B10409F0BFCF1F8E18A281E090E089A398
:1008C0009AA37E018FE1E80EF11C4E0193E2890E9E
:1008D000911C98E0792EF701A190B1907F0160E81A
:1008E000C801EEDE6C01892BA9F41E8E1D8E7C8E54
:1008F0001B8EA114B10469F1AA94AB2809F0B2CF00
:1009000064E224E0AE01455E5F4FC8018CDE8E14C8
:100910009F0409F7C601A296CDBFDEBFDF91CF913C
:100920001F910F91FF90EF90DF90CF90BF90AF900D
:100930009F908F907F90089568E0A6CF60E1A4CF4C
:1009400064E1A2CF60E0A0CF1B8E1C8E1E8E1D8E98
:10095000A4CF60E2D6CF2F923F924F925F926F92D8
:100960007F928F929F92AF92BF92CF92DF92EF923F
:10097000FF920F931F93CF93DF93CDB7DEB76397AB
:10098000CDBFDEBF7C018091143C9091153C092EB7
:10099000000CAA0BBB0BAF6FBF688093003C909319
:1009A000013CA093023CB093033C84E08093043C60
:1009B00083E08093083C81E08093093C86E080934B
:1009C0000A3C10920B3C4BE0942E5E0184E1A80E91
:1009D000B11C8091043C893008F08BC086E0E8E4CB
:1009E000FFE4DE011E9601900D928A95E1F73E012B
:1009F000EEE06E0E711CF301C190D1903F018601B3
:100A0000000F111FF801EC0DFD1DE25BF04B808023
:100A1000682DC70141DE83FD93C07090043CF8E06F
:100A2000F71508F466C08091003C9091013CA091BC
:100A3000023CB091033CAC01BD01442777FD4395D6
:100A4000552766277727242FAC01BD01442755275A
:100A50006627707422242A94322C422CFFE15F2EE8
:100A6000211106C022242A94E7E03E2E412C512C6D
:100A700082219321A421B521222309F453C08C8320
:100A80009B83CD01AA27BB27282F220F220F220FDD
:100A9000207E382F33703860232B2A8335E09695DB
:100AA00087953A95E1F78983872D452B462B472B70
:100AB00009F080648D83472D50E068E07CE3CE012F
:100AC000069631D225E0270D0C0D1D1DF801E25BC5
:100AD000F04BAE014F5F5F4F6181C701A4DD28E09D
:100AE00048E0682DC70186DD682DC701D5DD807718
:100AF00019F09A9491106DCF6396CDBFDEBFDF9150
:100B0000CF911F910F91FF90EF90DF90CF90BF900A
:100B1000AF909F908F907F906F905F904F903F909D
:100B20002F9008959C0193E0369527959A95E1F7CB
:100B300029838295880F807E8A831C821B82B4CF92
:100B40006A147B0409F057CFD4CF1F920F920FB6CF
:100B50000F9211248F939F93AF93BF938091103C7A
:100B60009091113CA091123CB091133C0196A11DB3
:100B7000B11D8093103C9093113CA093123CB09314
:100B8000133C81E08093A60ABF91AF919F918F9112
:100B90000F900FBE0F901F9018951F93CF93DF9368
:100BA000EC01162FABDA1883812F96DACE01DF9194
:100BB000CF911F91A8CBEDE7FCE384E0818381E333
:100BC0008083EEE3FCE31582148262E082E89CE31A
:100BD000E4DF63E081E89CE3E0DF68E080E89CE339
:100BE000DCDF69E08FE79CE3D8CF91E088ED84BF3C
:100BF0009093610080910206856080930206809147
:100C00000006816080930006809102068F7C8065DB
:100C1000809302061092E20582E08093E4059093AF
:100C2000030A8EEF8093270A8093260A80E8809338
:100C30002D0A80932B0A8093290A80932C0A809393
:100C40002A0A8093280A89E08093000A87E080932B
:100C5000E505E0E8FAE0C7E09EEF80E8D5E0C18373
:100C600094878587D0837096E03C2AE0F207B9F735
:100C70001092A10A8FE39FE18093AC0A9093AD0A92
:100C80008091A50A81608093A50A1092A00A8091A4
:100C9000A00A81608093A00A789430DA6AE070E05C
:100CA00080E090E004DB85E190E08093163C909337
:100CB000173C81E08093183C8093193C80931A3C48
:100CC00024E130E020931B3C30931C3C80931D3C7E
:100CD00080931E3C92E090931F3C23E130E02093F0
:100CE000203C3093213C8093223C8093233C93E032
:100CF0009093243C22E130E02093253C3093263C25
:100D00008093273C8093283C94E09093293C21E1F8
:100D100030E020932A3C30932B3C80932C3C8093F2
:100D20002D3CD0932E3C20E130E020932F3C30939B
:100D3000303C8093313C8093323C96E09093333C3E
:100D40002FE030E02093343C3093353C8093363CA8
:100D50008093373CC093383C2EE030E02093393C00
:100D600030933A3C80933B3C80933C3C88E08093BA
:100D70003D3C80916000806890E028ED24BF809326
:100D8000600082E89CE3FBDC82E89CE3DADC82E83A
:100D90009CE3F3DC81E89CE3F2DC81E89CE3D1DCBA
:100DA00081E89CE3EADC80E89CE3E9DC80E89CE302
:100DB000C8DC80E89CE3E1DC8FE79CE3E0DC8FE7C4
:100DC0009CE3BFDC8FE79CE3D8DCC6E1DCE38EE389
:100DD000E82E8CE3F82EEC16FD0651F0188119323E
:100DE00028F4812F79D960E0812FDAD92596F3CFC5
:100DF000F0910411809106117091081160910A110F
:100E000090910C11E091031120910511509107115F
:100E10004091091130910B11880F811D880F8F2788
:100E2000770F711D770F711D8727629560FB67959E
:100E300067F9862792959827822F880F811D880F42
:100E40008E27252F220F211D220F211D8227242FBF
:100E5000229520FB279527F98227232F2295822789
:100E60008093143C9093153C82E89CE374DD81E808
:100E70009CE371DD80E89CE36EDD8FE79CE36BDD36
:100E8000C0E0D0E082E89CE366DD68EE73E080E0DD
:100E900090E00DDA2097B1F3B3D8F4CF38D0A59F06
:100EA000900DB49F900DA49F800D911D1124089565
:100EB00097FD1094002E083098F00850232F342FFF
:100EC000452F562F672F782F892F912DF4CF15940A
:100ED0009795879577956795579547953795279572
:100EE0000A95AAF71124002D08950024A7FD009467
:100EF0002A173005400550056005700580059005EE
:100F00000895EE0FFF1F0590F491E02D0994A29F24
:100F1000B001B39FC001A39F01D0B29F700D811D8E
:100F20001124911D0895FB01DC0102C001900D9276
:0C0F300041505040D8F70895F894FFCFCE
:100F3C000000010002000300040005000000010095
:100F4C00020030313640414650515600000000003E
:100F5C00000000000000000005010101010101007A
:100F6C000000000000000000000000000000000075
:100F7C00000203000001020304050607000102033E
:100F8C000405000102030405060700010203040521
:100F9C00060700010203000102030405060000001D
:100FAC000000000000010101010101020202020225
:100FBC0002020203030303030303030404040405F2
:100FCC0005050505050501020408102040800102F5
:100FDC0004081020010204081020408001020408BB
:0F0FEC0010204080010204080102040810204078
:00000001FF
